:1000000002049F7FC87EF8DEFE00DFF92211031193
:100010000311031103110311031103110311031140
:1000200003DDEA227D01110DC2A011437D0A11FA00
:100030009005D47401119B9005E57402119B7D021B
:10004000110D2275A030115A75A030115A75A030CB
:10005000115A75A020115A118A22D2A01163C2A090
:100060001163227F05DFFE22F5A0C2A3115A3333AC
:100070003333F5A0C2A3115A22F5A0D2A3115A33EB
:10008000333333F5A0D2A3115A2274281168740CAB
:100090001168740611687401116822B4010C74802F
:1000A000116811C074801168800A74C0116811C091
:1000B00074C01168E493B40001221179A380F52281
:1000C000781874201179D8FA22748011687818741D
:1000D000201179D8FA74C0116878187420D8F022E9
:1000E00074801168781874201179D8FA2274C011BC
:1000F00068781874201179D8FA227E327F64DFFE86
:10010000DEFADDF622C0E0E5F024801168D0E011CF
:100110007922C0E0E5F024C01168D0E011792275A1
:10012000F00A842430C0F08535F03105D0F0E5F0D8
:10013000243005358535F031052275F00A842430E8
:10014000C0F08535F03112D0F0E5F024300535856A
:1001500035F03112227590FF7580FFC2B2E59085AF
:1001600080F0D2B2227590FFC2B2E590D2B222F5F1
:100170009085F080C2B100D2B122F590C2B100D218
:10018000B122D2A230A2FB2275A0B031652275A0A7
:100190009031652275A0B0317A2275A090317A2213
:1001A00075A0F0317A2275A01031552275A010315A
:1001B0006F2275A010317A2275A0D031652275A00A
:1001C000D0317A2275A03031652275A05031652278
:1001D00075A07031652275A0F03165220000000025
:1001E00031D620E7F72200000000110331D620E7C6
:1001F000F530E6F2220000000031D620E7F730E3C8
:10020000F4220000000031D620E7EA20E3E72231A3
:10021000A6DFFC2231D630E30431A680F72231A6D6
:1002200085F00E31A6F50F85F01022E50E75350527
:10023000313A743A75F0073112E50F753508313AE5
:100240002211967D0A11FA9005F67401119BC2B035
:100250001103D2B07D02110D31DC31B8C2E431BEE0
:1002600031DC318EB414073188B4EB02800280FE99
:10027000749031A031DC31C420E00280FE2231A62E
:10028000C5F01179E5F01179DEF42211967D0A119D
:10029000FA9006297401119B74C01168740231949C
:1002A000E4319A74A131A0318231A620E00820E126
:1002B00005750806800920E00630E1037508087F0F
:1002C0001A510F7E14517E511431E62278707F103E
:1002D000760008DFFB510274A031A02231F578705E
:1002E000AF08E608C0E0E608F5F0D0E031ACDFF298
:1002F000318231D62251CC75700051DCC330E0011F
:1003000022D32211967D0A11FA90065C7401119B8A
:1003100090066D7402119B30B3117A011103110321
:10032000110351F550F11ABA00F2221205ACE53C66
:10033000B471217D0A11FA90063A7401119B90065E
:100340004B7402119B51CC75701B7574037578004A
:1003500051DC80AF7D0A11FA90067E7401119B90EA
:10036000068F7402119B51CC75701B7574027578E1
:0E0370000051DC750C01808B74FF319A3194C2
:10037E0051CC757042757102757240757301757747
:10038E00FF7578FF51DC20E00420E30522751DFF88
:10039E002231A685F01D31A631A631A6F50BB50A80
:1003AE000280044002E509F50CE50B75350E311F90
:1003BE00511E74C01168511E512B51142211967486
:1003CE00FF319A319451CC7570437571027577FF78
:1003DE007578FF51DC20E00520E304D322C32231DF
:1003EE00A631A6F50985F00A7D0A11FA9006C274A7
:1003FE0001119B9006D37402119BE50975350B31E3
:10040E001FE50A75350E311FE50A04F51E31A631BA
:10041E00A6F50D511EE50E75350B313AE50F753506
:10042E000E313AE50DB50909850E14850F158510A7
:10043E0016B4AA09850E17850F18851019B50C0963
:10044E00850E1A850F1B85101C31DC20E3BFD322CD
:10045E0051CC75704E51DC227D0A11FA9006A074B3
:10046E0001119BE50C75350E311F900618740211A3
:10047E009B51CC75704785147385157485167585DB
:10048E00177685187785197851DC30E002C322D3B0
:10049E002275813FC2A0750C017511007512007591
:1004AE00130011245141518B7D01110D710371CB3C
:1004BE0050FA30B70530B37780F81196916650EC4C
:1004CE007D01110D7178E51DB41134E50EB5110CD9
:1004DE00E50FB51207E510B513028023850E1185C1
:1004EE000F12851013110330B63A30B34230B76293
:1004FE0030B40530B50E80CC915E750C0180AD75B3
:10050E000C01800BE50C14B40016850A0C800091CA
:10051E005E71CB5097851A14851B15851C16809A13
:10052E00F50C80EBE50C04B51EF6750C0180E09120
:10053E005E7D0A11FA90067E7401119B90068F74EF
:10054E0002119B51CC75701B75740251DC750C0138
:10055E0081BA7D0A11FA9006B17401119BE50C75F2
:10056E00350C311F51CC75704B75780051DC110371
:10057E001103110330B48130B70730B3B2110380C9
:10058E00F37D0A11FA9006A07401119B1103110359
:10059E00110351CC75704B75780151DC81EA7416DC
:1005AE00319A319451CC75705A757100757201750E
:1005BE0077FF7578FF51DC20E30380E22231A6310C
:1005CE00A6F53C5114222043442D526F6D20506CE1
:1005DE0061796572202000202056657273696F6EF6
:1005EE0020352E3120202000496E6974696E6720F7
:1005FE00202020202020202000202020202020200D
:10060E002020202020202020200054696D652020ED
:10061E00202020202020202020200020204964653A
:10062E006E74696679696E67202020002020204351
:10063E006C6F736520446F6F722020200020202085
:10064E0057616974696E672E2E2E2020200020209F
:10065E002052656164696E6720434420202000208B
:10066E00202057616974696E672E2E2E202020007F
:10067E002020204F70656E20446F6F722020202046
:10068E000020202057616974696E672E2E2E20205F
:10069E002000506C6179696E6720547261636B2023
:1006AE00202000506175736520547261636B2020A9
:1006BE0020202000547261636B52616E67652020AA
:1006CE00202D202000546F74616C2054696D6520BC
:1006DE0020203A20200052656164696E6720544FD5
:0E06EE004320202020200020506C65617365A1
:1006FC0020496E736572742020002020204175649F
:0B070C00696F204344202020202000C3
:00000001FF
